:100000003BC0E2C154C053C052C051C050C04FC0E9
:100010004EC04DC04CC04BC04AC049C048C047C08C
:1000200046C045C044C0040309041C0377007700A0
:1000300077002E00660069007300630068006C00A2
:100040002E00640065000E0355005300420061005D
:100050007300700012011001FF000008C016DC05DB
:1000600002010102000109021200010100801909C8
:10007000040000000000000011241FBECFE5D4E002
:10008000DEBFCDBF10E0A0E6B0E0EAEFFEE002C0C8
:1000900005900D92A236B107D9F710E0A2E6B0E0C4
:1000A00001C01D92A33AB107E1F7CDD424C7A8CF70
:1000B00085B7836085BF8BB780648BBF0895FF923F
:1000C0000F931F93CF93DF9360918700161654F51B
:1000D00080918400CCE0D0E0C81BD109C557DF4F28
:1000E0006350809183008D3279F08091620087FDAA
:1000F00011C0CE01B9D48F3F09F481C0882309F41F
:10010000A1C090E080E008C08AE58093610068307B
:1001100009F47BC090E880E09093620080936000D7
:10012000109287008091610084FF27C08091600059
:100130008F3F19F1182F893008F058C0811B809328
:1001400060008091620080FD28C02BE4F22E8F5F5A
:100150008093620087FD28C0112309F076C004E077
:1001600088E790E0612F2CD1183019F08FEF809341
:100170006000F0927700009361009AE080B3847190
:1001800031F49150D9F71092880010928200DF91DB
:10019000CF911F910F91FF90089593ECF92E8F5FEF
:1001A0008093620087FFD8CFC0918500D0918600F0
:1001B00086FD58C0112399F01150DE01E8E7F0E008
:1001C000412F50E01F5F9A0127583F4F8D91819337
:1001D000E217F307D9F74F5F5F4FC40FD51FD093D6
:1001E0008600C0938500012F0C5FBACF18E0811BF9
:1001F000809360008091620080FDCFCFA6CF8EE11A
:100200008093610090E08FEF87CF8881807609F03E
:1002100043C020E830E0109280008981882309F0F3
:1002200046C010928100309386002093850090E8AC
:1002300022E08F81882321F48E81821708F46CCF0D
:10024000822F6ACF90E08FEF67CF88E790E0612F31
:10025000ADD4182F893008F480C08FEF80936000F0
:100260000EE187CF112309F4BACF11509E01A8E700
:10027000B0E0612F70E01F5FAB0147585F4FF9019D
:1002800084918D932F5F3F4FA417B507C1F76F5F20
:100290007F4FC60FD71FA3CFCE01D8D4282F8F3FB3
:1002A00079F5888187FD10C08FEF90E035CF8530DC
:1002B00071F0863091F08830D1F0893019F18A30B0
:1002C00099F190E820E0B5CF8E8190E025CF8A812A
:1002D0008093880090E820E0ACCF8B818130A1F141
:1002E000823049F18330A1F090EC20E0A2CF8AE87F
:1002F00090E0909386008093850090E821E099CF6C
:1003000090E897CF8A8180938A0090E820E091CF8F
:100310008A81882329F586E290E090938600809375
:10032000850090EC24E085CF3093860020938500F3
:1003300090E821E07ECF86E690E09093860080935F
:10034000850090EC22E175CF84E590E090938600E3
:100350008093850090EC22E16CCF082F0C5F00CFDA
:10036000813061F0823009F0BFCF86E490E0909355
:1003700086008093850090EC2EE05BCF8AE290E0CF
:10038000909386008093850090EC2CE152CFA82FAB
:10039000B92F8FEF9FEF41E050EA615070F02D913F
:1003A00038E0722F782796958795269570FF02C0C2
:1003B000842795273A95A9F7F0CF809590950895D1
:1003C000E6DF8D939D930895CF93CFB7CF93849B12
:1003D000FECF849B09C0849B07C0849B05C0849B7F
:1003E00003C0849B01C09EC0DF93C0918400DD27C1
:1003F000C557DF4F849B02C0DF91EBCF2F930F9344
:100400001F9300B32FEF04FB20F94F933F9310B3DA
:100410004FEF012704FB21F93BE031C04E7F012F54
:1004200010B3216028C0102F4D7F2260000000B360
:1004300029C04B7F2460012F000010B32BC010B3E4
:10044000477F28602AC04F7E00B320612CC04F7DBB
:1004500010B320622FC04F7B00B3206432C042270C
:1004600000B349934FEF0000102714FB20F910B39D
:100470001471A9F1297F91F2012704FB21F900B33E
:10048000237F89F23150F0F1102714FB22F910B3C9
:10049000277E79F2012704FB23F92F7C81F200B338
:1004A000102714FB24F92F7971F200C010B3012733
:1004B00004FB25F92F7359F200C000B3102714FB79
:1004C00026F9223040F200C010B3012704FB27F9BF
:1004D000243028F64F77206810B30000F9CF3B5046
:1004E0003195333010E41ABFB8F0C31BD0400881F7
:1004F000033C41F10B3431F11981412F1F772091D9
:100500008200121731F4093691F10D3279F0013E73
:1005100069F02227209389003F914F911F910F91FD
:100520002F91DF91CF91CFBFCF9118950093890084
:100530003F914F911F910F912F91DF91CAB7C6FD47
:1005400046CFF0CF00918900002331F3109187004E
:10055000112349F534304AF130938700009383002A
:10056000109184003BE0311B309384001EC0009149
:1005700087000130C4F40AE53091610034FD17C0F2
:1005800000936100C7E7D0E016C0052710E002BB6A
:100590001FC0052722C0052727C005272CC0052717
:1005A00010E002BB33C04AE503C042ED01C0432F57
:1005B000C4E1D0E032E011B31461949A02B311BBEC
:1005C0005F9354E120E820FF052702BB279517958C
:1005D0001C3FD8F620FF0527279502BB17951C3F27
:1005E000C0F620FF05272795179502BB1C3F98F6FC
:1005F00020FF0527279517951C3F02BB70F600C00A
:10060000499120FF052702BB279517951C3F38F617
:1006100020FF0527279502BB17951C3F38F520FFC3
:1006200005272795179502BB1C3F10F520FF0527CE
:10063000279517951C3F02BBE8F4242F3A9519F62D
:100640000B7E5F9102BB00C010918800C651D04064
:1006500011F01093820010E41ABF006111B31B7EE9
:10066000402F4B7E02BB11BB42BB56CF0527D3CFD9
:100670000527D8CF0527DDCF82E58DB981E08EB97A
:100680000895882339F08CE993E09093A200809339
:10069000A10008958DE793E09093A2008093A100BC
:1006A000089592B782B7891B8C30E0F3089587B321
:1006B0008C6287BBC298C59892B782B7891B8C3071
:1006C000E0F3C29A92B782B7891B8C30E0F3C298EC
:1006D0008091A1009091A2008C59934009F0089557
:1006E00082E58DB981E08EB9089587B3837D87BB9C
:1006F00088B3837D88BB1DB80895482F30E020E083
:1007000047FD16C0C398330FB4993F5FC59A92B79F
:1007100082B7891B8C30E0F3C59892B782B7891BEA
:100720008C30E0F32F5F283029F0440F47FFEACFE9
:10073000C39AE9CF832F08958FB9779BFECF8FB1EE
:100740000895EF92FF920F931F930FE1E091A100A4
:10075000F091A20082E5F82EEE24E3948CEA09954C
:10076000E091A100F091A20083E50995E091A1003C
:10077000F091A20080E00995182FE091A100F0917E
:10078000A20080E00995133519F11DB8C59A92B7FA
:1007900082B7891B8C30E0F3C59892B782B7891B6A
:1007A0008C30E0F3E091A100F091A20083E0EC39FD
:1007B000F80721F0002331F00150D0CFFDB8EEB89A
:1007C0000023D1F781E01F910F91FF90EF900895E2
:1007D00080E01F910F91FF90EF900895EF92FF92AC
:1007E0000F931F937B018C01862F8170880F880FD8
:1007F000880FE091A100F091A20080620995D801D4
:10080000C70129E0B695A795979587952A95D1F7C1
:10081000E091A100F091A200099516950795F79433
:10082000E794E091A100F091A2008E2D0995E0914E
:10083000A100F091A20080E009951F910F91FF9017
:10084000EF9008950F931F938C01E091A100F09118
:10085000A20080EA0995E091A100F091A200812F09
:100860000995E091A100F091A200802F0995E091F7
:10087000A100F091A20080E009951F910F910895C9
:10088000FF920F931F938C01F62EE091A100F0913F
:10089000A20080EC0995E091A100F091A200812FC7
:1008A0000995E091A100F091A200802F0995E091B7
:1008B000A100F091A2008F2D09958EE1B7D080E0C4
:1008C0001F910F91FF900895CF92DF92EF92FF92C8
:1008D0000F931F936B017C01142FE091A100F09105
:1008E000A2008CE40995D701C60149E0B695A79509
:1008F000979587954A95D1F7E091A100F091A200D4
:100900000995D701C601B695A79597958795E0916A
:10091000A100F091A2000995E091A100F091A20040
:1009200080E009951F3FF1F012B70EE1C701B60153
:1009300055DF8F3F79F482B7811B8D33B8F312B73F
:100940000150A1F781E01F910F91FF90EF90DF9090
:10095000CF90089580E01F910F91FF90EF90DF906E
:10096000CF9008958FE062D080E01F910F91FF90AB
:10097000EF90DF90CF900895CF92DF92EF92FF92A9
:100980000F931F936B017C01042F122F862F817010
:10099000880F880F880FE091A100F091A200806479
:1009A0000995D701C60169E0B695A79597958795F2
:1009B0006A95D1F7E091A100F091A2000995D701C5
:1009C000C601B695A79597958795E091A100F091FE
:1009D000A2000995E091A100F091A200802F099555
:1009E0001123C1F00F37F1F012B70EE1C701B601C4
:1009F000F5DE8F3779F482B7811B8D33B8F312B7E8
:100A00000150A1F781E01F910F91FF90EF90DF90CF
:100A1000CF90089580E01F910F91FF90EF90DF90AD
:100A2000CF9008958FE002D080E0F5CF382F882353
:100A300049F020E092B782B7891B8C33E0F32F5F37
:100A40002317C0F308958B9893988B9A939A93E009
:100A500097BB94BB8EEF85BB93BF81E012DE28DB92
:100A600078942DDB2CDBFDCFFF920F931F93CF9358
:100A7000DF93F82E292F062F40916300413051F06B
:100A8000443041F01FEF812FDF91CF911F910F91E3
:100A9000FF900895002309F487C08F2D922F9C01A9
:100AA000E90110E053C08091730090917400892B8C
:100AB00009F058C060916F007091700080917100D2
:100AC00090917200488121E057DF809164009091FD
:100AD000650001979093650080936400892BD9F499
:100AE000109263008091750081FF3AC0809176007A
:100AF00090E020917300309174008217930781F188
:100B000060916F00709170008091710090917200FF
:100B10004881DADE11E080916F0090917000A09121
:100B20007100B09172000196A11DB11D80936F00FC
:100B300090937000A0937100B093720021969E0173
:100B40002F19201708F09FCF40916300413009F41E
:100B5000AACF80916F0090917000688191DEB5CF2F
:100B600011E0D9CF60916F00709170008091710099
:100B700090917200488120E0FFDE809176008150E4
:100B800080937600882309F0A0CF60916F00709168
:100B900070008091710090917200488195DE809183
:100BA00073008093760091CF10E06DCF0F931F9369
:100BB000CF93DF93082F162F40916300842F82502C
:100BC000823038F01FEF812FDF91CF911F910F916D
:100BD0000895662399F1802F9C01E90120C080913E
:100BE0006F00909170002EDE888380916F0090914D
:100BF0007000A0917100B09172000196A11DB11D0D
:100C000080936F0090937000A0937100B093720076
:100C100021969E01201B211778F4409163004230F9
:100C2000F1F660916F007091700080917100909169
:100C30007200D4DD8883D9CF183028F61092630073
:100C4000812FDF91CF911F910F9108950F931F93E3
:100C5000CF93DF938C01DC0111968C91813051F19F
:100C6000823009F4C2C0833089F1843009F491C024
:100C7000873009F462C0853009F436C1863009F442
:100C8000ECC0883009F4B7C0893081F481E08093EA
:100C90006600F80182819381A481B58180936F0001
:100CA00090937000A0937100B093720080E0C7E64B
:100CB000D0E037C09A9B3EC081E0E3DC1092660032
:100CC000C09AF5DC80E0C7E6D0E02BC0E091A1003F
:100CD000F091A200D80112968C910995C7E6D0E058
:100CE00080936700E091A100F091A200D8011396D3
:100CF0008C91099580936800E091A100F091A20089
:100D0000D80114968C91099580936900E091A10017
:100D1000F091A200D80115968C91099580936A00F4
:100D200084E0D0938600C0938500DF91CF911F911E
:100D30000F91089580E0A5DCC1CF809166008823E3
:100D400099F4F801938180E0228130E0822B932B8B
:100D5000AA2797FDA095BA2F80936F0090937000FB
:100D6000A0937100B0937200D80117969C911797C9
:100D700080E016962C9130E0822B932B90936500A7
:100D80008093640083E0809363008FEFC7E6D0E038
:100D9000C8CF80916600882399F4F801938180E0A0
:100DA000228130E0822B932BAA2797FDA095BA2FA2
:100DB00080936F0090937000A0937100B0937200C5
:100DC000D80117969C91179780E016962C9130E0E9
:100DD000822B932B909365008093640082E0809334
:100DE00063008FEFC7E6D0E09CCF7FDCC09880E047
:100DF000C7E6D0E096CF809166008823B1F4D80191
:100E000013969C91139780E012962C9130E0822BE0
:100E1000932BAA2797FDA095BA2F80936F009093EC
:100E20007000A0937100B093720010927400109241
:100E3000730010927500F801978180E0268130E000
:100E4000822B932B909365008093640084E08093C1
:100E500063008FEFC7E6D0E064CF809166008823FF
:100E600099F4F801938180E0228130E0822B932B6A
:100E7000AA2797FDA095BA2F80936F0090937000DA
:100E8000A0937100B0937200D80114968C911497BE
:100E900015969C91292F2F7020937500492F50E0B3
:100EA000407F507042955295507F5427407F542781
:100EB000480F511D509374004093730020FF02C0EF
:100EC00040937600F801978180E0268130E0822B04
:100ED000932B909365008093640081E0809363007E
:100EE0008FEFC7E6D0E01DCF2CDCC7E6D0E08093C3
:0A0EF000670081E016CFF894FFCFF1
:020EFA00FF5A9D
:00000001FF
